:100000000C942A000C9445000C9445000C94450077
:100010000C9445000C9491010C94BE010C94E601E3
:100020000C9445000C943D010C9445000C94450043
:100030000C9445000C9445000C9408030C94450066
:100040000C9445000C9445000C9445000C9445001C
:100050000C94450011241FBECFE5D4E0DEBFCDBF18
:1000600010E0A0E6B0E0E6E7FCE002C005900D92EB
:10007000A637B107D9F710E0A6E7B0E001C01D929E
:10008000AA3CB107E1F70C94A9000C940000CF93AF
:10009000DF93CDB7DEB7E7E3F0E08FE18083E4E301
:1000A000F0E08CEF8083E1E3F0E084E08083DF9197
:1000B000CF910895CF93DF93CDB7DEB721970FB6D9
:1000C000F894DEBF0FBECDBFF89480E29EE490931B
:1000D000C7008093C60019822FC08981482F5527F9
:1000E00089819927880F991FFC01E257FF4F808172
:1000F00091819C0128513C4FCA01880F991FFC0136
:10010000EA54FF4F318320832091C6003091C7000D
:1001100089819927880F991FFC01EA54FF4F80813C
:100120009181A901481B590BCA019093C700809384
:10013000C60089818F5F89838981883070F27894C5
:1001400021960FB6F894DEBF0FBECDBFDF91CF91E1
:100150000895CF93DF93CDB7DEB721970FB6F8940C
:10016000DEBF0FBECDBF0E9447000E941B010E9450
:10017000FA020E9449031092B50085EA92E090933A
:1001800089008093880083EF92E090938B008093A6
:100190008A00789480917A008823E1F310927A00A3
:1001A0000E94AF0500C080917C00813041F4109224
:1001B0007C008091B500882311F40E945A00809140
:1001C0007A00813081F710927A0019821CC080E693
:1001D00090E00E948303898199270E94CD0387E6DE
:1001E00090E00E94830389819927880F991FFC0161
:1001F000EA54FF4F808191810E94CD030E94BE038B
:1002000089818F5F89838981893008F3CCCFCF932F
:10021000DF93CDB7DEB7F894E9E5F0E089E18083BC
:100220007894DF91CF910895CF93DF93CDB7DEB768
:10023000DF91CF910895CF93DF93CDB7DEB7E3E59C
:10024000F0E082E08083EFE4F0E01082EEE4F0E0A2
:1002500082E08083EAE4F0E084EF91E091838083A0
:10026000E8E4F0E080ED97E091838083E9E5F0E059
:1002700089E18083DF91CF9108951F920F920FB68D
:100280000F9211248F93CF93DF93CDB7DEB7809178
:10029000B4008F5F8093B4008091B4008834C9F5B6
:1002A00081E080937B001092B40080917F008F5F8B
:1002B00080937F0080917F00853029F410927F0029
:1002C00081E080937C0080917D008F5F80937D0032
:1002D00080917D00843641F410927D0081E080930E
:1002E000780081E080937A0080917D00823319F458
:1002F00081E080937A0080917E008F5F80937E0002
:1003000080917E008A3029F410927E0081E08093F3
:100310007900DF91CF918F910F900FBE0F901F90BA
:1003200018951F920F920FB60F9211242F933F939F
:100330004F935F936F937F938F939F93AF93BF93ED
:10034000EF93FF93CF93DF93CDB7DEB7E0918800B3
:10035000F09189000995DF91CF91FF91EF91BF91C5
:10036000AF919F918F917F916F915F914F913F914D
:100370002F910F900FBE0F901F9018951F920F9204
:100380000FB60F9211248F93AF93BF93EF93FF9308
:10039000CF93DF93CDB7DEB7A2E3B0E0E2E3F0E0C6
:1003A00080818B7F8C93A8E3B0E0E8E3F0E080816C
:1003B0008F7E8C93DF91CF91FF91EF91BF91AF91A1
:1003C0008F910F900FBE0F901F9018951F920F9254
:1003D0000FB60F9211242F933F938F939F93AF9358
:1003E000BF93EF93FF93CF93DF93CDB7DEB7229701
:1003F000DEBFCDBFA2E3B0E0E2E3F0E08081846045
:100400008C93ECE4F0E011821082A8E4B0E08091DB
:1004100076009927880F991FFC01EA54FF4F8081CD
:10042000918111969C938E9380917600882339F464
:10043000A8E3B0E0E8E3F0E0808180618C938091F4
:100440007600282F33273A83298389819A81823045
:100450009105C1F129813A812330310554F4898114
:100460009A81009789F029813A8121303105D9F0AC
:100470004EC089819A818330910599F129813A8111
:1004800024303105E9F143C0A8E3B0E0E8E3F0E04F
:10049000808180618C93A8E3B0E0E8E3F0E08081A4
:1004A00081608C9334C0A8E3B0E0E8E3F0E08081A1
:1004B0008E7F8C93A8E3B0E0E8E3F0E08081826077
:1004C0008C9325C0A8E3B0E0E8E3F0E080818D7F65
:1004D0008C93A8E3B0E0E8E3F0E0808184608C9343
:1004E00016C0A8E3B0E0E8E3F0E080818B7F8C9356
:1004F000A8E3B0E0E8E3F0E0808188608C9307C077
:10050000A8E3B0E0E8E3F0E08081877F8C938091FE
:1005100076008F5F8093760080917600893010F0AE
:10052000109276002296F894DEBFCDBFDF91CF9176
:10053000FF91EF91BF91AF919F918F913F912F913B
:100540000F900FBE0F901F901895CF93DF93CDB7EC
:10055000DEB780918000909181000097B1F4E6E4CD
:10056000F0E0808191819093870080938600AEE4D3
:10057000B0E0EEE4F0E080818F7B8C9381E090E04E
:1005800090938100809380002BC0E6E4F0E08081AE
:1005900091819093850080938400AEE4B0E0EEE416
:1005A000F0E0808180648C932091840030918500FC
:1005B0008091860090918700A901481B590BCA01C0
:1005C00090938300809382001092810010928000AB
:1005D00080918200909183009093C9008093C8001D
:1005E000DF91CF910895CF93DF93CDB7DEB7DF9141
:1005F000CF910895CF93DF93CDB7DEB7E7E2F0E078
:100600001082E6E2F0E08FEE8083DF91CF910895D3
:100610001F920F920FB60F9211242F933F938F9337
:100620009F93EF93FF93CF93DF93CDB7DEB7E6E2CF
:10063000F0E01082809177009927E4E2F0E02081D9
:100640003181880F991FFC01E257FF4F31832083CE
:10065000809177008F5F809377008091770088305A
:1006600010F010927700E7E2F0E08091770080834D
:10067000E6E2F0E08FEE8083DF91CF91FF91EF9182
:100680009F918F913F912F910F900FBE0F901F90D0
:100690001895CF93DF93CDB7DEB7E9E2F0E080E1C4
:1006A0008083E0E4F0E01082EAE2F0E088E1808319
:1006B000E0E4F0E086E88083EBE2F0E082EC808327
:1006C000DF91CF910895CF93DF93CDB7DEB7219718
:1006D0000FB6F894DEBF0FBECDBF8983EBE2F0E02A
:1006E00080819927807290700097C1F3ECE2F0E06E
:1006F0008981808321960FB6F894DEBF0FBECDBFEF
:10070000DF91CF910895CF93DF93CDB7DEB72697D2
:100710000FB6F894DEBF0FBECDBF9E838D838D8153
:100720009E81DC01FD0101900020E9F73197CF01A6
:100730008A1B9B0B9C838B831A8219820FC0298191
:100740003A818D819E81F901E80FF91F80810E9415
:10075000630389819A8101969A83898329813A81E9
:100760008B819C818217930750F726960FB6F894D9
:10077000DEBF0FBECDBFDF91CF910895CF93DF9342
:10078000CDB7DEB7809169000E94630380916A0053
:100790000E946303DF91CF910895CF93DF93CDB78C
:1007A000DEB766970FB6F894DEBF0FBECDBF9E8B47
:1007B0008D8B8D899E894AE050E09E012F5F3F4FCF
:1007C000B9010E94F605CE0101960E948303669648
:1007D0000FB6F894DEBF0FBECDBFDF91CF91089565
:1007E000CF93DF93CDB7DEB722970FB6F894DEBF75
:1007F0000FBECDBF8A8387E089831FC08A81482FBF
:1008000055278981282F332727FD309581E090E0F7
:10081000022E02C0880F991F0A94E2F784239523C1
:100820001816190624F481E30E94630303C080E3D1
:100830000E94630389818150898389818823F4F62A
:10084000809169000E94630380916A000E946303A3
:1008500022960FB6F894DEBF0FBECDBFDF91CF91C9
:100860000895CF93DF93CDB7DEB726970FB6F894F0
:10087000DEBF0FBECDBF9E838D838EE190E09C8353
:100880008B831CC084E690E09A8389830EC08D819F
:100890009E8101979E838D838D819E810097B9F7FC
:1008A00089819A8101979A83898389819A810097A6
:1008B00099F78B819C8101979C838B838B819C8191
:1008C000009701F726960FB6F894DEBF0FBECDBF96
:1008D000DF91CF910895CF93DF93CDB7DEB7219706
:1008E0000FB6F894DEBF0FBECDBF898389819927EB
:1008F00081709070882341F0A5E3B0E0E5E3F0E07B
:10090000808180618C9307C0A5E3B0E0E5E3F0E06F
:1009100080818F7E8C938981992782709070009757
:1009200041F0A5E3B0E0E5E3F0E0808180628C93E4
:1009300007C0A5E3B0E0E5E3F0E080818F7D8C9314
:100940008981992784709070009741F0A5E3B0E009
:10095000E5E3F0E0808180648C9307C0A5E3B0E01C
:10096000E5E3F0E080818F7B8C9389819927887003
:100970009070009741F0A5E3B0E0E5E3F0E08081FE
:1009800080688C9308C0A5E3B0E0E5E3F0E09081D7
:100990008FE789238C9321960FB6F894DEBF0FBEA4
:1009A000CDBFDF91CF910895CF93DF93CDB7DEB761
:1009B000A5E3B0E0E5E3F0E0808184608C9381E022
:1009C00090E00E943104A5E3B0E0E5E3F0E080812F
:1009D0008B7F8C93DF91CF910895CF93DF93CDB729
:1009E000DEB722970FB6F894DEBF0FBECDBF8A8365
:1009F0008A8182958F70898389810E946B040E940D
:100A0000D4048A810E946B040E94D40422960FB6FB
:100A1000F894DEBF0FBECDBFDF91CF910895CF9385
:100A2000DF93CDB7DEB721970FB6F894DEBF0FBEC8
:100A3000CDBF8983A5E3B0E0E5E3F0E08081886085
:100A40008C9389810E94ED0421960FB6F894DEBF45
:100A50000FBECDBFDF91CF910895CF93DF93CDB778
:100A6000DEB724970FB6F894DEBF0FBECDBF9C83D0
:100A70008B838B819C81DC01FD0101900020E9F7D3
:100A80003197CF018A1B9B0B8A8319820EC0898103
:100A900099279C018B819C81F901E80FF91F8081C6
:100AA0000E940F0589818F5F898399818A819817B8
:100AB00070F324960FB6F894DEBF0FBECDBFDF9162
:100AC000CF910895CF93DF93CDB7DEB721970FB6BF
:100AD000F894DEBF0FBECDBF898381E090E00E9415
:100AE0003104A5E3B0E0E5E3F0E08081877F8C93FB
:100AF00089810E94ED04A5E3B0E0E5E3F0E08081A8
:100B000088608C9321960FB6F894DEBF0FBECDBFE0
:100B1000DF91CF910895CF93DF93CDB7DEB72397C1
:100B20000FB6F894DEBF0FBECDBF8A836B838A8178
:100B3000882319F48B81805889838A81813019F444
:100B40008B818054898389810E94620523960FB628
:100B5000F894DEBF0FBECDBFDF91CF910895CF9344
:100B6000DF93CDB7DEB781E090E00E943104A5E3CA
:100B7000B0E0E5E3F0E08081877F8C9383E00E9422
:100B80006B040E94D40485E090E00E94310483E06D
:100B90000E946B040E94D40481E090E00E94310422
:100BA00083E00E946B040E94D40482E00E946B04E4
:100BB0000E94D40481E090E00E94310488E20E9407
:100BC00062058EE00E94620581E00E9462058BE66C
:100BD00090E00E942D056AE081E00E948B0580E78D
:100BE00090E00E942D05DF91CF910895FB019F01B8
:100BF000E8944230C4F04532B4F44A3029F497FB0B
:100C00001EF4909581959F4F642F77270E942706A9
:100C1000805D8A330CF0895D8193CB010097A1F749
:100C200016F45DE251931082C9010C941706DC01A1
:100C3000FC0101900020E9F73297AE17BF0730F4AE
:100C40007C916081708331976D93F7CF0895AA1BD3
:100C5000BB1B51E107C0AA1FBB1FA617B70710F0A7
:100C6000A61BB70B881F991F5A95A9F780959095D9
:060C7000BC01CD01089556
:100C76004B2000000000003D000D0A6875687500F5
:060C8600416B6B750000DC
:00000001FF
